:100000000C942A001895000018950000189500001F
:10001000189500001895000018950000189500002C
:100020001895000018950000189500000C948504A0
:10003000189500000C94A0120C94D2121895000090
:1000400018950000189500001895000018950000FC
:10005000189500008FE58DBFCCEFECE44E2E88E0C4
:100060008EBFD7E0F7E05F2EEEEFF7E0A0E6B0E05E
:10007000A89584B7082E877F84BF88E1992781BD22
:1000800091BD88278D933197E9F788E089B980E0A1
:1000900080BD88E18AB9662480E08ABB80E087BBA6
:1000A000BC9ABB9ABA9A8FEF84BB8FEF81BB8A98B8
:1000B00087E886B980E087B9379A85E083BF81EB0E
:1000C0008FBD81E08EBD8FEF8ABD579A0E94C91304
:1000D000A7E4B1E0ECE9F7E20E94E010A9E4B1E0A6
:1000E000EEE9F7E20E94E010ABE4B1E0E0EAF7E20B
:1000F0000E94E010AFE4B1E0E4EAF7E20E94E01011
:10010000A3E5B1E0E8EAF7E20E94E010A7E5B1E07C
:10011000ECEAF7E20E94E010ABE5B1E0E0EBF7E2D9
:100120000E94E010AFE5B1E0E4EBF7E20E94E010DE
:10013000A3E6B1E0E8EBF7E20E94E010A7E6B1E049
:10014000ECEBF7E20E94E010ABE6B1E0E0ECF7E2A6
:100150000E94E010AFE6B1E0E4ECF7E20E94E010AC
:10016000A3E7B1E0E8ECF7E20E94E010A7E7B1E016
:10017000ECECF7E20E94E01081E080937B0182E0EA
:1001800080937C0183E080937D0184E080937E01F5
:1001900085E080937F0186E08093800187E08093F3
:1001A000810188E08093820189E0809383018AE065
:1001B000809384018BE0809385018CE0809386019D
:1001C0008FEF8ABD80E088BD00E218ED2CE03FE0B3
:1001D000ACE9B1E00D931D932D933C9380E08093A7
:1001E000CE0184E690E0A4EEB1E08D939C93C29A98
:1001F00086E990E00E94A410C39A86E990E00E94EC
:10020000A410C49A8AEF90E00E94A410C298C398E8
:10021000C49880E090E0A2E9B1E08D939C9301E066
:1002200010E020E030E0A8EAB1E00D931D932D939B
:100230003C934AE050E060E070E0A8EAB1E00D9144
:100240001D912D913C910E9403131CF011F00C9410
:100250004901A2E9B1E00D911C910F931F9307B1E1
:10026000007E076007B90E94E610482F592F1F91A2
:100270000F91040F151FA2E9B1E00D931C9381E0CB
:1002800090E00E94A410A8EAB1E00E94500F0C94E4
:100290001901A2E9B1E00D911C914AE050E00E94E1
:1002A000730FA2E9B1E04D935C9384E690E00E9465
:1002B000A410A2E9B1E00D911C91043650E015079D
:1002C0000CF402C00C94690184E08093E6010C9464
:1002D0004E0A80E090E0A3EDB1E08D939C9301E0A5
:1002E00010E020E030E0A8EAB1E00D931D932D93DB
:1002F0003C934AE050E060E070E0A8EAB1E00D9184
:100300001D912D913C910E9403131CF011F00C944F
:10031000A901A3EDB1E00D911C910F931F9307B1BB
:10032000007E066007B90E94E610482F592F1F91E2
:100330000F91040F151FA3EDB1E00D931C9381E005
:1003400090E00E94A410A8EAB1E00E94500F0C9423
:100350007901A3EDB1E00D911C914AE050E00E94BB
:10036000730FAEEDB1E04D935C9384E690E00E9494
:10037000A41000E010E020E030E0ACE8B1E00D9324
:100380001D932D933C9301E010E020E030E0A8EABB
:10039000B1E00D931D932D933C934AE050E060E053
:1003A00070E0A8EAB1E00D911D912D913C910E9461
:1003B00003131CF011F00C941A0207B1007E0560C3
:1003C00007B90E94E610A4EAB1E08D939D938827B7
:1003D0008D938C9300E014E020E030E0A4EAB1E0DB
:1003E0004D915D916D917C910E94FE12A4EAB1E065
:1003F0000D931D932D933D93ACE8B1E00D911D91AC
:100400002D913C91A4EAB1E04D915D916D917C916B
:100410000E94F912ACE8B1E00D931D932D933D932A
:1004200085E090E00E94A410A8EAB1E00E94500F7D
:100430000C94CD01ACE8B1E00D911C914AE050E084
:100440000E94990FA2EEB1E04D935C9304EF11E08E
:1004500020E030E0A2EEB1E04D915C916627772775
:100460000E94BD10A8E9B1E00D931D932D933D931B
:1004700000E010E020E030E0A8E8B1E00D931D932B
:100480002D933C9301E010E020E030E0A8EAB1E0D9
:100490000D931D932D933C934AE050E060E070E093
:1004A000A8EAB1E00D911D912D913C910E9403139A
:1004B0001CF011F00C94870207B1007E036007B9AD
:1004C0000E94E610A4EAB1E08D939D9388278D9356
:1004D0008C93A8E8B1E00D911D912D913C91A4EA77
:1004E000B1E04D915D916D917C910E94F912A8E867
:1004F000B1E00D931D932D933D9385E090E00E9414
:10050000A410A8EAB1E00E94500F0C944C02A8E895
:10051000B1E00D911C914AE050E00E94990FA0EECD
:10052000B1E04D935C93A0EEB1E00D911C910039C8
:1005300051E0150710F00C94A20283E08093E601CD
:100540000C944E0AA0EEB1E00D911C91083552E0DA
:10055000150718F011F00C94AF020C94B40283E06C
:100560008093E6010C944E0AA2EEB1E00D911C912D
:100570000E3551E0150710F00C94C30282E0809311
:10058000E6010C944E0AA2EEB1E00D911C910E3ED4
:1005900052E0150718F011F00C94D0020C94D5021B
:1005A00082E08093E6010C944E0A789489B78160CA
:1005B00089BF00913B01013011F00C940D0380E0E4
:1005C00080933B01A6EBB0E03FE30E94BC0FA6EB9B
:1005D000B0E08C91082F0A3011F00C940B03A6EBBD
:1005E000B0E00E94AF13082F41E0041BACE3B1E080
:1005F0000C93A6EBB0E00E94AF13EA2FFB2F009103
:100600003C013197E01BF0400FEFA6EBB0E00E94F9
:10061000A7130C94E7020E94500C00914601013090
:1006200011F00C94C5038BE10E940B10E0EDF7E292
:100630000E9401108BE10E940B10E6EDF7E20E9490
:100640000110EAEDF7E20E9401100E940810E2EFAB
:10065000F7E20E9401100E940810EAE0F8E20E940E
:100660000110A4E3B7E0E0EBF1E00E9419130E944F
:10067000F90F0E940810E6E1F8E20E940110A4E3DD
:10068000B7E0E6ECF1E00E9419130E94F90F0E9416
:100690000810E0E2F8E20E940110A4E3B7E0E3ED05
:1006A000F1E00E941E130E94F90F0E940810ECE274
:1006B000F8E20E940110A4E3B7E0E2E9F1E00E9451
:1006C0001E130E94F90F0E940810ECE3F8E20E944A
:1006D0000110A4E3B7E0E0E9F1E00E941E130E94DC
:1006E000F90F0E940810EAE4F8E20E940110A4E366
:1006F000B7E0E4EBF1E00E941E130E94F90F0E94A4
:100700000810EAE5F8E20E940110A4E3B7E0E6EB86
:10071000F1E00E941E130E94F90F0E940810ECE6FF
:10072000F8E20E940110A4E3B7E0EAECF1E00E94D5
:1007300019130E94F90F0E940810E6E7F8E20E94E0
:100740000110A4E3B7E0E6EEF1E00E9425130E9459
:10075000F90F0E940810E2E8F8E20E940110A4E3F9
:10076000B7E0EEECF1E00E9425130E94F90F0E9421
:100770000810ECE8F8E20E9401100E94081088ECD2
:1007800090E00E94A4100C94830484E190E00E9405
:10079000A410E0E9F8E20E940110A4E3B7E0E0EB66
:1007A000F1E00E9419130E94F90F0E94081084E1E1
:1007B00090E00E94A410E6E9F8E20E940110A4E390
:1007C000B7E0E6ECF1E00E9419130E94F90F0E94D5
:1007D000081084E190E00E94A410ECE9F8E20E9485
:1007E0000110A4E3B7E0E3EDF1E00E941E130E94C4
:1007F000F90F0E94081084E190E00E94A410E2EA40
:10080000F8E20E940110A4E3B7E0E2E9F1E00E94FF
:100810001E130E94F90F0E94081084E190E00E94CC
:10082000A410E8EAF8E20E940110A4E3B7E0E0E9CE
:10083000F1E00E941E130E94F90F0E94081084E14B
:1008400090E00E94A410EEEAF8E20E940110A4E3F6
:10085000B7E0E4EBF1E00E941E130E94F90F0E9442
:10086000081084E190E00E94A410E4EBF8E20E94FA
:100870000110A4E3B7E0E6EBF1E00E941E130E9432
:10088000F90F0E94081084E190E00E94A410EAEBA6
:10089000F8E20E940110A4E3B7E0EAECF1E00E9464
:1008A00019130E94F90F0E94081084E190E00E9441
:1008B000A410E0ECF8E20E940110A4E3B7E0E6EE39
:1008C000F1E00E9425130E94F90F0E94081084E1B4
:1008D00090E00E94A410E6ECF8E20E940110A4E36C
:1008E000B7E0EEECF1E00E9425130E94F90F0E94A0
:1008F000081084E190E00E94A410ECE8F8E20E9465
:1009000001100E9408100C94D9020F921F922F928E
:100910003F924F925F927F92AF92BF920F931F933D
:100920002F933F934F935F936F937F938F939F93F7
:10093000AF93BF93CF93DF93EF93FF938FB78F93D3
:1009400083E4809352000E94810A0E9416060E944E
:100950004E050E94F2060E94C9048F918FBFFF913D
:10096000EF91DF91CF91BF91AF919F918F917F9147
:100970006F915F914F913F912F911F910F91BF9078
:10098000AF907F905F904F903F902F901F900F906F
:100990001895A4EBB1E00D911C91043B50E01507B4
:1009A0001CF011F00C94D6040C94DC0484EB90E061
:1009B000A4EBB1E08D939C93A4EBB1E00D911C915D
:1009C0000C345FEF15070CF402C00C94ED048CE4BA
:1009D0009FEFA4EBB1E08D939C93A6EBB1E00D915A
:1009E0001C91043B50E015071CF011F00C94FA0424
:1009F0000C94000584EB90E0A6EBB1E08D939C9302
:100A0000A6EBB1E00D911C910C345FEF15070CF4CF
:100A100002C00C9411058CE49FEFA6EBB1E08D931E
:100A20009C93A4EBB1E00D911C91003050E01507B0
:100A30000CF402C00C941F05969A0C94200596980D
:100A4000A6EBB1E00D911C91003050E015070CF4BD
:100A500002C00C942E05979A0C942F059798A4EB3E
:100A6000B1E08D919C910E94930FA0EAB1E08D932B
:100A70009C93A6EBB1E08D919C910E94930FA2EA0A
:100A8000B1E08D939C930FEF4091A001041B0ABD30
:100A9000A2EAB1E08C9188BD08950895A0EBB1E081
:100AA0000D911D912D913C91A8EAB1E00D931D93FC
:100AB0002D933C93A8EAB1E00D911D912D913C91AD
:100AC00041E150E060E070E00E94BD10A8EAB1E0B2
:100AD0000D931D932D933D93A6ECB1E00D911D91C7
:100AE0002D913C9141E150E060E070E00E94BD102A
:100AF000A4EAB1E00D931D932D933D93A4EAB1E0D8
:100B00000D911D912D913C91A8EAB1E04D915D911F
:100B10006D917C910E94F912AAECB1E00D931D93A6
:100B20002D933D93AFECB1E00D911D912D913C9132
:100B3000AAECB1E04D915D916D917C910E94F9120A
:100B4000AFECB1E00D931D932D933D9348ED56ED21
:100B500060E070E0AFECB1E00D911D912D913C9102
:100B60000E9403131CF011F00C94B8050C94C205FC
:100B700008ED16ED20E030E0AFECB1E00D931D93F1
:100B80002D933C9348E259E26FEF7FEFAFECB1E079
:100B90000D911D912D913C910E9403130CF402C004
:100BA0000C94DC0508E219E22FEF3FEFAFECB1E067
:100BB0000D931D932D933C93AFECB1E00D911D91DE
:100BC0002D913C914BE950E060E070E00E943C10B8
:100BD000A8EAB1E04D935D936D937D93AAECB1E0EB
:100BE0000D911D912D913C9145EA50E060E070E03F
:100BF0000E943C10A4EAB1E04D935D936D937D9308
:100C0000A8EAB1E00D911D912D913C91A4EAB1E0CB
:100C10004D915D916D917C910E94F912AAEBB1E02A
:100C20000D931D932D933D930895089500E010E0DA
:100C300020E030E0A4EAB1E00D931D932D933C93A6
:100C400040E050E060E070E0AFECB1E00D911D914C
:100C50002D913C910E9403131CF011F00C9432066C
:100C60000C944406AFECB1E00D911D912D913C9197
:100C700040E25EE460E070E00E94FE12A4EAB1E0AF
:100C80000D931D932D933D93A4EAB1E00D911D9119
:100C90002D913C9146E450E060E070E00E943C10F1
:100CA000A4EAB1E04D935D936D937D9380E090E075
:100CB000A7EEB1E08D939C934DE050E060E070E0D2
:100CC000A4EAB1E00D911D912D913C910E94031376
:100CD0001CF011F00C946E060C9478060DE010E0F8
:100CE00020E030E0A4EAB1E00D931D932D933C93F6
:100CF00040E050E060E070E0A4EAB1E00D911D91A9
:100D00002D913C910E9403130CF402C00C949206A6
:100D100000E010E020E030E0A4EAB1E00D931D9384
:100D20002D933C9340E050E060E070E0A4EAB1E035
:100D30000D911D912D913C910E9403131CF011F017
:100D40000C94A4060C94AF06A4EAB1E08D919C919A
:100D5000A7EEB1E08D939C9382E080938701009190
:100D60008701003011F00C94F00648EA54EB67E07C
:100D700070E0ACE9B1E00D911D912D913C910E9484
:100D800003131CF011F00C94C7060C94CA06C29A07
:100D9000C398C49848EA54EB67E070E0ACE9B1E06E
:100DA0000D911D912D913C910E9403130CF402C0F2
:100DB0000C94DD06C39AC498C29848E55EE667E0E5
:100DC00070E0ACE9B1E00D911D912D913C910E9434
:100DD00003130CF402C00C94F006C398C298C49A92
:100DE00008950895A8EBB1E00E945F0FA8EBB1E071
:100DF0000D911C910A3050E015071CF011F00C9475
:100E000003070C94130700918701013011F00C9433
:100E10000C07C29AC39AC49A00918701023011F05C
:100E20000C941307C49AA8EBB1E00D911C9100310A
:100E300050E015071CF011F00C9420070C944607A5
:100E400000918701003018F011F00C9429070C94E0
:100E50003107C298C398C498A5EDB1E08C918F5F1B
:100E60008C9381E090E0A8EBB1E08D939C9300918E
:100E7000D5010A3018F011F00C9440070C94460785
:100E800080E08093D50180E080938701AEEDB1E0F2
:100E90000D911D9117FB1EF42FEF3FEF02C022278B
:100EA0003327A3EDB1E04D915D9157FB1EF46FEF39
:100EB0007FEF02C0662777270E94FE12AAEDB1E0FD
:100EC0000D931D932D933D93AFECB1E00D911D91CA
:100ED0002D913C9140E25EE460E070E00E943C10A5
:100EE000A4EAB1E04D935D936D937D93A4EAB1E0E4
:100EF0000D911D912D913C910E949010A4EAB1E0BA
:100F00000D931D932D933D9341E050E060E070E020
:100F1000A4EAB1E00D911D912D913C910E94031323
:100F20000CF402C00C949E0701E010E020E030E0D9
:100F3000A4EAB1E00D931D932D933C93AAEDB1E08B
:100F40000D911D912D913C91A4EAB1E04D915D91DF
:100F50006D917C910E943C10AAEDB1E04D935D93A0
:100F60006D937D93AFECB1E00D911D912D913C916E
:100F700040ED57E060E070E00E943C10A4EAB1E070
:100F80004D935D936D937D93A4EAB1E00D911D9116
:100F90002D913C910E949010A4EAB1E00D931D9315
:100FA0002D933D9346E150E060E070E0A4EAB1E0AB
:100FB0000D911D912D913C910E9403131CF011F095
:100FC0000C94E4070C94EE0706E110E020E030E01A
:100FD000A4EAB1E00D931D932D933C930BE110E037
:100FE00020E030E0A4EAB1E04D915D916D917C91FB
:100FF0000E94FE12A4EAB1E00D931D932D933D9340
:10100000A4EAB1E00D911D912D913C914FEF5FEF5E
:101010006FEF7FEF0E94BD10ACEAB1E00D931D931E
:101020002D933D93A4EAB1E04D915D916D917C913A
:10103000AAEDB1E00D911D912D913C910E940313F9
:101040001CF011F00C9426080C943208A4EAB1E0CC
:101050000D911D912D913C91AAEDB1E00D931D9341
:101060002D933C93ACEAB1E04D915D916D917C91F3
:10107000AAEDB1E00D911D912D913C910E940313B9
:101080000CF402C00C945008ACEAB1E00D911D9133
:101090002D913C91AAEDB1E00D931D932D933C93BE
:1010A000AAEDB1E00D911D912D913C91AEEBB1E017
:1010B0000D931D932D933C930027A0E3B0E08C91FA
:1010C00082FB0EF401E040E0041711F00C9470086C
:1010D0008DE790E0A4EEB1E08D939C930C948A0888
:1010E000A4EEB1E00D911C91003355E715070CF407
:1010F00002C00C948708A4EEB1E00D911C9141E070
:1011000050E0040F151FA4EEB1E00D931C9381E095
:1011100080938701AAEBB1E00D911D912D913C9137
:101120004DE750E060E070E00E94BD10AAEBB1E036
:101130000D931D932D933D93AAEBB1E00D911D915D
:101140002D913C91A4EEB1E04D915D9157FB1EF4C1
:101150006FEF7FEF02C0662777270E943C10AAEB53
:10116000B1E04D935D936D937D93AAEBB1E00D914A
:101170001C91AEEBB1E04D915C91041B150BA4EBFF
:10118000B1E00D931C93AAEBB1E00D911C91AEEB75
:10119000B1E04D915C91040F151FA6EBB1E00D93EA
:1011A0001C930091CE01003011F00C943B0980E0BB
:1011B00090E0A4EBB1E08D939C9380E090E0A6EBEF
:1011C000B1E08D939C9300E010E020E030E0AAEBCA
:1011D000B1E00D931D932D933C9300E010E020E0CF
:1011E00030E0A2ECB1E00D931D932D933C9300E011
:1011F00010E020E030E0AFECB1E00D931D932D93B3
:101200003C9300E010E020E030E0A4E9B1E00D9371
:101210001D932D933C9300E010E020E030E0A0EB24
:10122000B1E00D931D932D933C9300E010E020E07E
:1012300030E0A6EDB1E00D931D932D933C93A2E910
:10124000B1E00D911C91023350E015071CF011F034
:101250000C942C090C94390981E08093CE0100E0B4
:1012600010E020E030E0A6EDB1E00D931D932D934A
:101270003C930C944C0A013011F00C94BD09A2E986
:10128000B1E00D911C91023350E015070CF402C03F
:101290000C94BB0940E050E060E070E0AFECB1E0DE
:1012A0000D911D912D913C910E9403130CF402C0ED
:1012B0000C94710940E050E060E070E0AFECB1E008
:1012C0000D911D912D913C910E9403130CF402C0CD
:1012D0000C94710981E080938701A6EDB1E00E9432
:1012E000500F40E050E060E070E0AFECB1E00D91F5
:1012F0001D912D913C910E9403131CF011F00C9450
:1013000083090C949C0940E050E060E070E0AFEC91
:10131000B1E00D911D912D913C910E9403131CF0A1
:1013200011F00C9495090C949C0981E0809387013D
:10133000A6EDB1E00E94500F40E550E060E070E0A3
:10134000A6EDB1E00D911D912D913C910E940313EA
:101350001CF011F00C94AE090C94BB0983E080934F
:10136000CE0100E010E020E030E0A6EDB1E00D930A
:101370001D932D933C930C944C0A033011F00C9464
:10138000490A01E010E020E030E0A4EAB1E00D936A
:101390001D932D933C934FEF50E060E070E0A4EA82
:1013A000B1E00D911D912D913C910E9403131CF011
:1013B00011F00C94440AA4EBB1E00D911C910030A3
:1013C00050E0150781E009F080E08F93A6EBB1E0D3
:1013D0000D911C91003050E0150781E009F080E08C
:1013E0009F918923882311F40C94F8090C94440AE2
:1013F000A4EBB1E00D911C91003050E015071CF0FA
:1014000011F00C94050A0C94090AA4EBB1E00E94B7
:10141000660FA4EBB1E00D911C91003050E0150770
:101420000CF402C00C94180AA4EBB1E00E945F0F08
:10143000A6EBB1E00D911C91003050E015071CF0B7
:1014400011F00C94250A0C94290AA6EBB1E00E9435
:10145000660FA6EBB1E00D911C91003050E015072E
:101460000CF402C00C94380AA6EBB1E00E945F0FA6
:1014700082E390E00E94A4100E94C904A4EAB1E0B3
:101480000E94500F0C94CB0980E08093CE010C9405
:101490004C0A83E08093CE010895089501E010E0A6
:1014A00020E030E0A8EAB1E00D931D932D933C932A
:1014B000A6EEB1E04C91552766277727A8EAB1E060
:1014C0000D911D912D913C910E9403131CF011F080
:1014D0000C947A0AC49A86E990E00E94A410C498F9
:1014E00086E990E00E94A410A8EAB1E00E94500FA3
:1014F0000C94580AE2E0F0E00E9433100C944E0A7B
:10150000089507B1007E056007B90E94E610ACE8B7
:10151000B1E08D939D9388278D938C9300E014E028
:1015200020E030E0ACE8B1E04D915D916D917C91AF
:101530000E94FE12ACE8B1E00D931D932D933D93F4
:1015400007B1007E036007B90E94E610A8E8B1E089
:101550008D939D9388278D938C9307B1007E0060B7
:1015600007B90E94E610A0E9B1E08D939C9307B102
:10157000007E066007B90E94E610A3EDB1E08D93EE
:101580009C9300E014E00F931F9307B1007E076067
:1015900007B90E94E610482F592F1F910F91041B85
:1015A000150BA2E9B1E00D931C93A4E9B1E00D91F4
:1015B0001D912D913C9144EF51E060E070E00E945C
:1015C0003C10A8EAB1E04D935D936D937D93A4E93F
:1015D000B1E00D911D912D913C91A8EAB1E04D91A2
:1015E0005D916D917C910E94FE12A4E9B1E00D9392
:1015F0001D932D933D93A8E8B1E00D911D912D9180
:101600003C91A0EEB1E04D915C91662777270E9456
:10161000FE12A8EAB1E00D931D932D933D93A8EA25
:10162000B1E00D911D912D913C91A7EEB1E04D914E
:101630005D9157FB1EF46FEF7FEF02C0662777279F
:101640000E94F912A8EAB1E00D931D932D933D93EA
:10165000A4E9B1E00D911D912D913C91A8EAB1E072
:101660004D915D916D917C910E94F912A4E9B1E0D8
:101670000D931D932D933D93A8E9B1E00D911D911C
:101680002D913C9144EF51E060E070E00E943C10ED
:10169000A4EAB1E04D935D936D937D93A8E9B1E029
:1016A0000D911D912D913C91A4EAB1E04D915D9178
:1016B0006D917C910E94FE12A8E9B1E00D931D93FB
:1016C0002D933D93A8E9B1E00D911D912D913C9191
:1016D000ACE8B1E04D915D916D917C910E94F91261
:1016E000A8E9B1E00D931D932D933D93A8E9B1E0D6
:1016F0000D911D912D913C9142E350E060E070E02E
:101700000E943C10A4EAB1E04D935D936D937D93EC
:10171000ACE8B1E00D911D912D913C914AE050E073
:1017200060E070E00E94BD10A8EAB1E00D931D9347
:101730002D933D93A4EAB1E00D911D912D913C9123
:10174000A8EAB1E04D915D916D917C910E94FE12ED
:10175000A4EAB1E00D931D932D933D93A4EAB1E06B
:101760000D911D912D913C9143E250E060E070E0BD
:101770000E94BD10A4EAB1E00D931D932D933D93FB
:10178000A4EAB1E00D911D912D913C9144E650E009
:1017900060E070E00E943C10A4EAB1E04D935D93DC
:1017A0006D937D93A4EAB1E00D911D912D913C9133
:1017B000A6ECB1E00D931D932D933C93A4E9B1E009
:1017C0000D911D912D913C91A6ECB1E04D915D9153
:1017D0006D917C910E94F912A4E9B1E00D931D93E3
:1017E0002D933D93A4E9B1E00D911D912D913C9174
:1017F00042E350E060E070E00E943C10A0EBB1E0FA
:101800004D935D936D937D93ACE9B1E00D911D9186
:101810002D913C9144EF51E060E070E00E943C105B
:10182000A4EAB1E04D935D936D937D93ACE9B1E093
:101830000D911D912D913C91A4EAB1E04D915D91E6
:101840006D917C910E94FE12ACE9B1E00D931D9365
:101850002D933D93ACE9B1E00D911D912D913C91FB
:10186000A0E9B1E04D915D9157FB1EF46FEF7FEF62
:1018700002C0662777270E94F912ACE9B1E00D9308
:101880001D932D933D930895089581E080933B012E
:101890000895A6EBB0E00E94FB0F0E940810089587
:1018A000A6EBB0E08C91082F033211F00C945C0C85
:1018B0000E94490C0C94D90CA6EBB0E08C91082F37
:1018C0000B3111F00C94680C0E94490C0C94D90C4B
:1018D000A6EBB0E0ECE9F7E22FEF91E00E94F41004
:1018E000A5E4B1E00C9300914501003018F011F02F
:1018F0000C947C0C0C94C90CA6EBB0E0ECECF8E278
:101900002FEF91E00E94F410002F003080E010F0E3
:1019100009F081E08F9340914501A6EBB0E0ECEC3B
:10192000F8E22FEF91E00E94F410002F041781E0FD
:1019300008F080E09F918923882311F40C94A80C6F
:101940000E94490C0E94DA0C0C94D90C0C94C70C20
:10195000E6EBF0E000914501A6EFB0E00E94A7138E
:10196000A6EFB0E00E946F13ADE3B1E00C930091DD
:101970003D01003011F00C94C30C0E94DA0C0C9461
:10198000D90C0C94C70C0E94490C0C94D90C0C94E3
:10199000D90C00913D01003011F00C94D50C0E943F
:1019A000DA0C0C94D90C0C94D90C0E94490C0C94B0
:1019B000D90C089581E08093EA01A6EFB0E0882772
:1019C0008C93A6E3B1E088278C93A0E4B1E0E8E92A
:1019D000F7E20E948C1280E090E0AEE3B1E08D93DC
:1019E0009C93A6EBB0E00E94AF13082F0F93A6EBD9
:1019F000B0E0E7E4F1E0222791E00E94F410402FEC
:101A00000F91041BA5E4B1E00C93A6EBB0E00E949B
:101A1000AF13EA2FFB2F009145013197E01BF040F7
:101A20000FEFA6EFB0E00E94A71381E08093E901D9
:101A30000091E901043018F011F00C94930D81E449
:101A4000482FA9EEB1E0AD90BB24A5EFB0E0AA0D00
:101A5000BB1D0C91041781E008F480E08F938AE5A8
:101A6000482FA9EEB1E0AD90BB24A5EFB0E0AA0DE0
:101A7000BB1D0C91041781E010F009F080E09F91EC
:101A800089238F9381E6482FA9EEB1E0AD90BB2466
:101A9000A5EFB0E0AA0DBB1D0C91041781E008F47E
:101AA00080E09F91892B8F938AE7482FA9EEB1E0C0
:101AB000AD90BB24A5EFB0E0AA0DBB1D0C9104179F
:101AC00081E010F009F080E09F918923882311F4D0
:101AD0000C948B0DA9EEB1E0AD90BB24A5EFB0E066
:101AE000AA0DBB1D8C91AAEEB1E0AD90BB24A5E37D
:101AF000B1E0AA0DBB1D8C93AAEEB1E08C918F5F73
:101B00008C9380E0AAEEB1E0AD90BB24A5E3B1E0F8
:101B1000AA0DBB1D8C93A9EEB1E08C918F5F8C93C5
:101B200010F40C94180DA6E3B1E00E94AF13082F37
:101B3000033011F00C94D70DE6E3F1E0A6E3B1E039
:101B40000E94941280E08093E9010091E90109313B
:101B500018F011F00C94D70DE9EEF1E00191112786
:101B600044E050E00E94B310E7E4F1E0E00FF11F21
:101B7000A6E3B1E00E94B71311F00C94CF0DA9EECB
:101B8000B1E0AD90BB24AAE7B1E0AA0DBB1D8C91DA
:101B9000AEE3B1E08D9388278C930C94D70DA9EE1A
:101BA000B1E08C918F5F8C9310F40C94A50D81E0C3
:101BB0008093EA01A6E3B1E088278C93A6EFB0E01A
:101BC000E9E4F1E0222791E00E94F410A5E4B1E0FD
:101BD0000C9300914501003011F00C94F60DA6EF26
:101BE000B0E00E94AF13A5E4B1E08C9381E0809354
:101BF000E901409145010091E901041718F011F045
:101C00000C94510E80E3482FA9EEB1E0AD90BB24B7
:101C1000A5EFB0E0AA0DBB1D0C91041781E008F4FC
:101C200080E08F9389E3482FA9EEB1E0AD90BB240B
:101C3000A5EFB0E0AA0DBB1D0C91041781E010F0D8
:101C400009F080E09F918923882311F40C94490EB8
:101C5000A9EEB1E0AD90BB24A5EFB0E0AA0DBB1D8D
:101C60008C91AAEEB1E0AD90BB24A5E3B1E0AA0D42
:101C7000BB1D8C93AAEEB1E08C918F5F8C9380E0BA
:101C8000AAEEB1E0AD90BB24A5E3B1E0AA0DBB1D67
:101C90008C93A9EEB1E08C918F5F8C9310F40C942F
:101CA000F90DAEE3B1E00D911C910F931F93A6E3E4
:101CB000B1E00E946F13402F512F1F910F91040F1D
:101CC000151FAEE3B1E00D931C93A6EFB0E0E9E47D
:101CD000F1E0222791E00E94F410002F003018F06C
:101CE00011F00C94750E0C947C0E809144018F774A
:101CF000809344010C94810E80914401806880930C
:101D00004401A6EFB0E00E94AF13082F0F93A6EF97
:101D1000B0E0E9E4F1E0222791E00E94F410402FC6
:101D20000F91041BA5E4B1E00C93A6EFB0E00E9474
:101D3000AF13EA2FFB2F009145013197E01BF040D4
:101D40000FEFA6EFB0E00E94A713A6EFB0E00E944D
:101D5000B811EDE0F0E0A0E4B1E00E94A113AEE321
:101D6000B1E00D911C91013050E0150711F00C9479
:101D7000D30EA6EBB0E0EEECF8E20E94E010A6EB8A
:101D8000B0E00E94B30FE8E8F1E00E941913A6EB5F
:101D9000B0E00E94B30FE6EDF8E20E94E0100E946E
:101DA000490C0C944F0F023050E0150711F00C94C1
:101DB000F30EA6EBB0E0E8EDF8E20E94E010A6EB2F
:101DC000B0E00E94B30FECE8F1E00E941913A6EB1B
:101DD000B0E00E94B30FE6EDF8E20E94E0100E942E
:101DE000490C0C944F0F033050E0150711F00C9480
:101DF000030FA6EBB0E0E0EEF8E20E94E0100E94D4
:101E0000490C0C944F0F043050E0150711F00C945E
:101E10001C0F81E0809346018BE10E940B10E0EDE6
:101E2000F7E20E9401108BE10E940B10E6EDF7E251
:101E30000E9401100C944F0F053050E0150711F06F
:101E40000C94270F80E0809346010C944F0F0630CE
:101E500050E0150711F00C94470FA6EBB0E0ECE052
:101E6000F9E20E94E010A6EBB0E00E94B30FE0E9B7
:101E7000F1E00E941E13A6EBB0E00E94B30FE6ED66
:101E8000F8E20E94E0100E94490C0C944F0FA6EB60
:101E9000B0E0E4E1F9E20E94E0100E94490C0895EC
:101EA0000D911D912D913C9181E0080F8827181FFD
:101EB000281F381F3C932E931E930E930895ED9187
:101EC000FC91EF5FFF4FFC93EE930895ED91FC9131
:101ED000E150F040FC93EE93089509D00E94B310B6
:101EE00000FC10D0089503D024D001F8F9CF0024CD
:101EF000E89457FF02C009D0689400F80BD010F89E
:101F00000124089502D009D00895509540954F5F5F
:101F10005F4F0895E89417FF0895009510950F5F9F
:101F20001F4F6894089599231AF48095909501960F
:101F30000895352F242FE894452B11F468940895C3
:101F4000512F402F0027112780E1440F551F001FFC
:101F5000111F021B130B416018F4020F131F4E7F59
:101F60008A9599F708958F938D918823E9F71197B2
:101F70008F910895A4E3B7E018D0883091F08D30A8
:101F800039F03323C9F38D933A9563FE44D0F4CFEF
:101F900063FC04C08DE03FD08AE03DD088278C935D
:101FA000089539D011973395E7CF0F929F93AF9350
:101FB000BF937F9380918A008823E1F3F894809106
:101FC0008A008A9580938A0090918800A0E6B0E00C
:101FD000A90F0024B01D8C919395983209F499278C
:101FE0009093880078947F91BF91AF919F910F90CB
:101FF0000895A4E3B7E08D91882311F00CD0FBCFB6
:1020000008950E94B411802D11F005D0FACF0895E3
:102010008DE001D08AE09F939FB79F93AF93BF93CA
:102020000F937F939091B5009832E1F3F8949091DB
:10203000B50093959093B50099270091B400ABE853
:10204000B0E0A00FB91F8C930395083209F4002764
:102050000093B400559A7F910F91BF91AF919F91DA
:102060009FBF9F91089588EE93E06ED03197D9F786
:10207000089500FC05D0089530D005D001F8F9CFBF
:1020800037D03FD00895842F952FA62FB72FE894EF
:10209000452B462B472B11F468940895402F512F60
:1020A000622F732F0027112722273327F0E2440FD6
:1020B000551F661F771F001F111F221F331F081B8C
:1020C000190B2A0B3B0B416028F4080F191F2A1F1C
:1020D0003B1F4E7FFA9559F708950024E89477FF47
:1020E00002C006D0689400F809D010F801240895C1
:1020F00012D04F5F5F4F6F4F7F4F0895E89437FFC7
:10210000089500951095209530950F5F1F4F2F4F24
:102110003F4F689408954095509560957095089547
:1021200037FF089500951095209530950F5F1F4F4C
:102130002F4F3F4F08953197F1F70895689462F853
:102140000895E89462F80895EF93FF93EE27E82B43
:10215000E92B31F0E0EAFFE03197F1F70197D1F791
:10216000FF91EF9108950F92B801469F8001479F1C
:10217000100D569F100D0F9008950F921F922F92E1
:10218000C801D901489F80014A9F90014B9F202C94
:10219000499F100D211D321D5A9F202C589F100D54
:1021A000211D321D599F200D311D689F200D311DAD
:1021B000699F300D789F300D2F901F900F900895DC
:1021C0000E94B4110D920020D9F70895369A3699DD
:1021D000FECF369A3699FECF84B195B10895999184
:1021E0000027A90FB01F1197492F4A955E2F6F2F17
:1021F000E89411274395203019F0C895802D01C02F
:1022000080818823B9F07C917723A1F0781739F485
:102210000EF0042F1395689411963196EBCF11238D
:1022200021F0411BA11B1127B10BE894E52FF62FDC
:102230001196E0CF882311F0002708950895D190DA
:10224000E190F19001910895219131914191519145
:102250000895102F90E8FF0C001F0927990FF7949D
:102260001078652F90E8440F551F5927990F47950F
:10227000607800380895FF0C90E89027110F97952B
:10228000F794092F0895502F2D2D3E2D4F2D612F9E
:1022900008952DEC3CEC4CEC5DE366270FC0CFDFDE
:1022A000F2DFDD24EE2490E8F92E0FE307C0CCDF47
:1022B00005C02227332740E251E46627552351F118
:1022C000002381F1C6DF71F1162700585058089499
:1022D000050B18F407FD03C025C007FD23C0469574
:1022E00037952795F694E794D79422D0FF202AF0CB
:1022F000DD0CEE1CFF1C015073F09D2D969548F0EF
:10230000DD203AF4EE202AF491E0D90E9927E91E57
:10231000F91EB1CF07C09FE7092FF92A9FEFD92EE9
:10232000E92E0895DD24EE24FF24002711270895C7
:102330009F929924AA24BB2488E1D216E306F406CE
:1023400028F0D21AE30AF40A089401C08894991C70
:10235000AA1CBB1CDD0CEE1CFF1C8A9571F7D92C46
:10236000EA2CFB2C9F900895C89531960020089583
:102370000E94A110E89488278A938A93D3DF1127BB
:102380008D918032E9F31197BBD098F08D3229F40A
:10239000109511968C91B4D060F08E3229F411967C
:1023A0008C91AED008F446C022960E949E1081E027
:1023B00008958C91A5D0D8F547D01196D0F7039504
:1023C0008D919ED0E0F38E3229F48C9199D010F447
:1023D0001196FBCF853419F0853609F055C011965A
:1023E0008C918ED060F08D3219F08B3221F0DCCFE1
:1023F00008800094088211968C9182D0A8F68053B0
:10240000898311968C917CD058F49981990F990FFA
:102410000980900D990F8053890F8983873220F6A8
:102420008981988199230AF48195080F2DC08E32F5
:1024300089F611968C9164D068F606D018F0119642
:102440000A95F8CF1196C1CF4F2D3E2D2D2DDD0CC5
:10245000EE1CFF1CA8F0DD0CEE1CFF1C88F0D20E59
:10246000E31EF41E68F0DD0CEE1CFF1C48F08053E8
:1024700009F06894D80E8827E81EF81E08F0089521
:10248000F42EE32ED22E089534D019F116F50983D7
:1024900008E921D00695882787959F2D9F77980F6B
:1024A000F92E0150000F110F07958981882379F0CB
:1024B0001AF48195898306C0ECDE89818A95898327
:1024C000D9F705C0F6DE89818A958983D9F72296E6
:1024D000089528DFFCCF0DD041F0FF2032F00A959F
:1024E00031F0DD0CEE1CFF1CD2F78894089508949F
:1024F000089500240D280E280F28002A0020089592
:10250000803320F08A3310F4089408958894089555
:1025100091E005C092E003C094E001C098E024DFA0
:102520000D929A95E1F70895819104D08D938823B7
:10253000D9F70895813618F08B3708F48F7D089508
:102540007F930F93AF93BF938F939F938FB78F9387
:10255000E89480918A0008E2081B21F49CB10E9453
:102560009E1013C000918900A0E6B0E077279CB1CF
:10257000A00FB71F9C936894839580938A0003955E
:10258000083209F40027009389009D3011F40E945D
:10259000450C8F918FBF9F918F91BF91AF910F91FC
:1025A0007F9118957F93AF93BF938F939F938FB72E
:1025B0008F939091B500992399F09A959093B500D7
:1025C0009927ABE8B0E08091B300A80FB91F9C91A8
:1025D0008395883209F488278093B3009CB901C0A1
:1025E00055988F918FBF9F918F91BF91AF917F91A0
:1025F0001895040F151F261F371F0895041B150B70
:10260000260B370B0895041715072607370708957B
:10261000000F111F221F331F08950095109520955C
:1026200030950F5F1F4F2F4F3F4F0895019110813D
:102630000EC001911191219130810BC00191108147
:1026400017FF05C03FEF2FEF04C00081112722279D
:10265000332737FF03C0E1DF8DE28D93CF93DF9304
:10266000CF92DF92EF92AA24BB24CC24DD24EE2467
:1026700040E2CAE0DD2755E093E38881890F87FDBA
:102680009F7083FD907F891B89935A95A9F7C0DFBE
:10269000AA1CBB1CCC1CDD1CEE1C4A9551F7E8940F
:1026A000EFE0FF2782910ED0EB30E0F71EF0689448
:1026B0008A2D0CD088278D93EF90DF90CF90DF91FB
:1026C000CF910895982F829501D0892F8F70805DCA
:1026D00026F0803309F4089568948D9308950027B7
:1026E0001127222733271DD08A3328F4803318F08E
:1026F00005D015D0F9CF0EF490CF089580538F9365
:10270000402F512F622F732F83DF82DF72DF80DF34
:102710008F919927080F191F291F391F08958D912F
:102720000895E894FCDF8032E9F38B32D9F38930E5
:10273000C9F38D3211F46894F2CF089588278D93F0
:10274000089594E081918D939A95E1F70895819190
:102750008D930A9519F08823D1F70895EFCF8FEF65
:1027600083959D919923E1F70895689401C0E894B9
:10277000AF93BF938D9116F0919103C00E94B41155
:10278000902D891718F011F48823A1F7BF91AF910C
:102790000895689463F80895000000003A003D0031
:1027A000414458004944470049444E0054454C00B8
:1027B0005354500053574900424154004D4F41007B
:1027C0004D4F420053545200455252004D4F440069
:1027D0005B313B3166005B324A002354656C656DAA
:1027E00065747269652076312E30202020202020EB
:1027F0000000232020202020202020202020202016
:1028000020202020202020200000234E65696775AD
:102810006E67203D2000234779726F203D20000025
:10282000234C656E6B6572203D200000234675DFEA
:10283000736368616C746572203D2000234261748B
:102840007465726965203D200000234D6F746F72BE
:10285000206C696E6B73203D2000234D6F746F7286
:1028600020726563687473203D20000023537472E6
:1028700065DF203D2000234665686C6572203D20A1
:102880000000234D6F647573203D2000313A340001
:10289000323A313D0000323A333D0000323A353DA4
:1028A0000000323A363D0000323A373D0000323AFD
:1028B000383D0000323A393D0000323A31303D00B7
:1028C000323A31313D00323A31323D002A00233074
:1028D0003A4144583D00210023303A4944473D00E5
:1028E00023303A49444E3D5B4350552D4D6F64753E
:1028F0006C2076332E3120626574612047FC6E7443
:102900006572204765726F6C645D210023303A4226
:1029100041543D0023303A4552523D5B53796E7429
:0C2920006178204572726F725D2100002A
:00000001FF
